:100000000C947F000C94F5010C949C000C949C00C3
:100010000C949C000C949C000C949C000C949C00F0
:100020000C949C000C949C000C949C000C949C00E0
:100030000C949C000C949C000C949C000C949C00D0
:100040000C949C000C949C000C949C000C949C00C0
:100050000C949C000C949C000C949C000C949C00B0
:100060000C949C000C949C00320349006E007400B8
:1000700065006C006C00690076006900730069001F
:100080006F006E00200063006F006E00740072004D
:100090006F006C006C006500720018037200610054
:1000A000700068006E00650074002E006E00650030
:1000B0007400040309040A033100300030003800E2
:1000C00005010905A1010901A10009300931150047
:1000D00026FF00750895028102C00509190129183B
:1000E00015002501750195188102C012010101005A
:1000F0000000089B282400030101020301001124D1
:100100001FBECFEFD4E0DEBFCDBF12E0A0E0B1E074
:10011000EAE1FBE002C005900D92A038B107D9F7E3
:1001200022E0A0E8B2E001C01D92A13DB207E1F7D4
:100130000E94DA040C948B050C940000CF93C62F18
:100140002091000124FF0BC02091A70238E823274B
:100150002093A702FC01A8EAB2E08C2F04C02AE594
:1001600020930001F7CF815018F091919D93FBCF20
:100170006C2F88EA92E00E94F101CC5FC0930001ED
:10018000CF910895CF93DF938091B70218160CF0AA
:10019000AEC09091B4022091B3022D3219F090E8D4
:1001A00080E09FC02AE5209301018B30C1F7CCE0AD
:1001B000D0E0C91BD109C554DD4F8881807609F094
:1001C00080C01092A502898181110BC01092A602F5
:1001D00085EA92E09093B6028093B50290E882E0BF
:1001E00079C0853021F48A818093B80271C086304D
:1001F00009F04BC08B81813009F442C0823021F478
:10020000CE010E94580360C0833069F58A81811154
:1002100009C082EB90E09093B6028093B50290EC17
:1002200084E058C0813049F48AE990E09093B602A6
:100230008093B50290EC88E14DC0823049F488E6A5
:1002400090E09093B6028093B50290EC82E342C0B6
:100250008330E1F586EB90E09093B6028093B5028F
:1002600090EC8CE037C0813249F483E992E09093BE
:10027000B6028093B50290EC89E02CC0823231F551
:10028000CE010E94580390EC25C0883019F48AEB07
:1002900092E00AC0893021F48A818093BA0218C0A2
:1002A0008A3049F485EA92E09093B6028093B502D1
:1002B00090E881E00FC08B3059F483EC8093A70263
:1002C00007C0CE010E94860390E804C090EC01C0F4
:1002D00090E880E02F81211104C02E81281708F4B6
:1002E000822F90938002809302011092B702809136
:1002F000010184FF46C0809102018F3F09F441C093
:10030000C82F893008F0C8E08C1B8093020120912F
:10031000800220FD02C0DBE401C0D3EC2F5F2093FC
:1003200080028091B5029091B60226FD05C0FC01C5
:10033000ADE9B2E02C2F0AC0ADE9B2E0FC012C2FF0
:10034000215048F034913D933196FACF215018F066
:1003500031913D93FBCF8C0F911D9093B60280930A
:10036000B5026C2F8DE992E00E94F10184E08C0FC0
:10037000C83019F09FEF90930201D0939C028093B4
:1003800001018AE099B1957031F48150D9F710924A
:10039000B8021092B202DF91CF910895E9E6F0E041
:1003A000808183608083E89A83EC8093A70208951C
:1003B000A82FB92F8FEF9FEF41E050EA615070F006
:1003C0002D9138E0722F782796958795269570FFA6
:1003D00002C0842795273A95A9F7F0CF809590958C
:1003E0000895E6DF8D939D930895CF93CFB7CF9374
:1003F000489BFECF489B09C0489B07C0489B05C04F
:10040000489B03C0489B01C09EC0DF93C091B402CB
:10041000DD27C554DD4F489B02C0DF91EBCF2F9302
:100420000F931F9309B12FEF00FB20F94F933F93D8
:1004300019B14FEF012700FB21F93BE031C04E7F9E
:10044000012F19B1216028C0102F4D7F22600000BC
:1004500009B129C04B7F2460012F000019B12BC0C6
:1004600019B1477F28602AC04F7E09B120612CC096
:100470004F7D19B120622FC04F7B09B1206432C07B
:10048000422709B149934FEF0000102710FB20F9D4
:1004900019B11570A9F1297F91F2012700FB21F90B
:1004A00009B1237F89F23150F0F1102710FB22F9B6
:1004B00019B1277E79F2012700FB23F92F7C81F205
:1004C00009B1102710FB24F92F7971F200C019B17E
:1004D000012700FB25F92F7359F200C009B110273D
:1004E00010FB26F9223040F200C019B1012700FBB1
:1004F00027F9243028F64F77206819B10000F9CF8A
:100500003B503195333011E01CBBB8F0C31BD040D9
:100510000881033C41F10B3431F11981412F1F77E0
:100520002091B202121731F4093691F10D3279F0AF
:10053000013E69F022272093B9023F914F911F910C
:100540000F912F91DF91CF91CFBFCF91189500934D
:10055000B9023F914F911F910F912F91DF91CCB331
:10056000C0FD46CFF0CF0091B902002331F31091C6
:10057000B7021123A1F53430A2F13093B7020093F2
:10058000B3021091B4023BE0311B3093B40229C096
:100590000091B70201301CF50AE547FD09C0309112
:1005A000010134FD20C000930101CCE9D2E01FC05D
:1005B0003091000134FD17C000930001C7EAD2E07A
:1005C00016C0052710E00BB91FC0052722C005275C
:1005D00027C005272CC0052710E00BB933C04AE51A
:1005E00003C042ED01C0432FC4E1D0E032E01AB1B4
:1005F0001560589A0BB11AB95F9355E020E820FFB7
:1006000005270BB9279517951C3FD8F620FF05271E
:1006100027950BB917951C3FC0F620FF0527279596
:1006200017950BB91C3F98F620FF052727951795BE
:100630001C3F0BB970F600C0499120FF05270BB98C
:10064000279517951C3F38F620FF052727950BB9EE
:1006500017951C3F38F520FF0527279517950BB9EF
:100660001C3F10F520FF0527279517951C3F0BB958
:10067000E8F4242F3A9519F60A7F5F910BB900C070
:100680001091B802C651D04011F01093B20211E09F
:100690001CBB01601AB11A7F402F4A7F0BB91AB9EF
:1006A0004BB94BCF0527D3CF0527D8CF0527DDCFB3
:1006B000FC018081807641F59181963031F59381FE
:1006C0009230D1F0923269F09130F9F480918B023E
:1006D00090918C029093B6028093B50280918A0229
:1006E000089580918E0290918F029093B60280932C
:1006F000B50280918D02089583E091E09093B60257
:100700008093B50282E2089580E0089522E832E005
:100710003093B6022093B502FC012081207620326E
:1007200099F48181813081F4E0918802F09189020D
:100730000088F189E02D82E892E00995E091880235
:10074000F09189028081089580E00895009741F03A
:1007500025E0E7E9F2E0DC0101900D922A95E1F74E
:1007600085E0E7E9F2E0A2E9B2E001900D928A9516
:10077000E1F7089524B1217C24B925B12E6325B970
:1007800018B820E227B92FE128B9E7EBFBE0319751
:10079000F1F700C0000026B120952F712A3150F4E6
:1007A00030E0F901EA59FD4F4081F901E45BFD4F6A
:1007B000208102C020E040E0FC014083FB01208357
:1007C0000895FF920F931F93CF93DF9300D000D033
:1007D000CDB7DEB7BE016F5F7F4FCE0102960E949C
:1007E000BA0387B1817E87B988B18E6188B985B136
:1007F000877C85B984B1886384B987EB9BE00197D6
:10080000F1F700C0000026B1269588B1817E88B935
:1008100087B18E6187B985B1877C85B984B1877CC2
:1008200084B985B1886385B9E7EBFBE03197F1F7CF
:1008300000C0000083B186958695869580952095A9
:100840008770F0E18F9FC00111242F70822B419798
:100850008A35910560F4FC01EE0FFF1FE856FE4F4C
:1008600000811181FC01E25CFE4F808104C080E0C8
:1008700090E000E010E018B817B82FEF28B915B8CD
:1008800028E024B925B1206325B9E7EBFBE03197D7
:10089000F1F700C0000023B124FF046025FF0160D0
:1008A00015B820E124B92D9AE7EBFBE03197F1F779
:1008B00000C000001D9B0260F82E9801287F232BAA
:1008C00021F0809191028C8315C0BE016D5F7F4F36
:1008D000CE0104960E94BA039C818A81981721F068
:1008E000809191028C8302C0909391029B818981B7
:1008F000981721F0809190028B8302C09093900210
:100900002C819FE3299F202D1124205820939702AA
:100910008B81899F902D1124905890939802009379
:10092000990210939A02F0929B020F900F900F90F1
:100930000F90DF91CF911F910F91FF900895CF936A
:10094000CFB7F89417B814B88FEF88B985B90E945B
:10095000E103CFBFCF9108958091250190912601A9
:10096000892B31F0109226011092250181E0089523
:1009700045E050E062E972E087E992E00E947E057E
:1009800008958E5F853038F4E82FF0E0E75CFE4F85
:10099000808190E0089580E890E0089580EC90E0F8
:1009A00090932C0180932B0187E291E0089582E1DE
:1009B00090E0089581E084B98EEF85B917B88FEF84
:1009C00088B988EF8BB985E08AB982E08093B0005E
:1009D00087E08093B10084EC8093B300209A84B1C7
:1009E000897F84B985B1866085B928980E94CE0434
:1009F000FC01909389028093880284819581909371
:100A00008F0280938E02828180938D0280859185F2
:100A1000009731F090938C0280938B02868108C0FE
:100A20008BEE90E090938C0280938B020E94D7040F
:100A300080938A0280918D0280931C018BB18A7F02
:100A40008BB98AB185608AB987EC9FEA0197F1F783
:100A500000C000008AB18A7F8AB9E0918802F091D3
:100A600089020284F385E02D09950E94CE017894D5
:100A700011E0D0E0C2E0A8950E94C200112341F02D
:100A8000E0918802F09189020484F585E02D0995B2
:100A9000B99B16C0C7BBD11115C0E0918802F09177
:100AA00089020484F585E02D0995E0918802F09192
:100AB00089020684F785E02D0995811103C01CC0C9
:100AC000DD23D1F08091000184FD03C0D1E010E06E
:100AD000D2CFE0918802F09189020088F189E02D5F
:100AE00082E892E00995E0918802F09189026081A4
:100AF00082E892E00E949E00D0E0E9CFFB01DC0199
:100B000004C08D910190801921F441505040C8F7E4
:0A0B1000881B990B0895F894FFCF9D
:100B1A005A5AFF090222000101008032090400002A
:100B2A00010300000009210101000122000007055C
:100B3A00810308000A010005002B000000000000E4
:100B4A00009F04E103AC04A603004080C0FF00003C
:100B5A00000001000000000000000000000000008A
:100B6A000000020000000000000000000000000079
:100B7A00000020000000001000000000000000003B
:100B8A000000040000000000000000000000000057
:100B9A0000008000000000000000000000000000CB
:100BAA0000004000000000080010000200004000A1
:100BBA000000000000000800000000000000000023
:100BCA000000000000000000002000040000800077
:100BDA0000000000000010000000000000000000FB
:100BEA0000000000000000000000000000000000FB
:100BFA0000000000000000000000000000000000EB
:100C0A000000000000000000004000080000000191
:100C1A0000000000000020000000000000000000AA
:100C2A0000000000000000000000000000000000BA
:100C3A00000000000000000000000808000000009A
:100C4A00000000000000000000000000000000009A
:100C5A00000000000000000000000000000000FF8B
:100C6A00FEFEFEFE00010000FFFE0000020201027D
:100C7A000000000002020000FEFE0001FFFE020268
:100C8A0000000202000000FFFEFE00000000010258
:00000001FF
